:020000040800F2
:10000000D81A0020CD000008493200084512000827
:1000100000000000000000000000000000000000E0
:10002000000000000000000000000000ED3C00089F
:100030000000000000000000E93200081D42000836
:10004000DF00000800000000DF000008DF000008FB
:10005000DF000008DF000008DF000008DF00000804
:1000600000000000DF000008AD0400084D05000896
:10007000DF000008DF000008DF00000800000000CB
:10008000DF0000082943000800000000DF0000082E
:10009000DF000008DF000008DF000008DF000008C4
:1000A000DF000008D13C0008DF00000841430008E1
:1000B000C94300080348854600F0D6F800480047C9
:1000C000FD4C0008D81A00200844F0470448804737
:1000D00004480047FEE7FEE7FEE7FEE7FEE7FEE72F
:1000E000CD420008B500000830B50B46014600209F
:1000F0002022012409E00D46D5409D4205D31D462E
:100100009540491B2546954040191546521E002D25
:10011000F1DC30BD70B500242546002801DA012449
:100120004042002901DA01254942FFF7DDFFAC42D8
:1001300000D04042002C00D0494270BDF8B50024E8
:100140002546002904DA0E46012400214042B1412F
:10015000002B04DA1E46002352420125B34100F071
:1001600052F88C4617461E46AC4203D0002540424A
:100170008D41AC46002C02D0002657429E4161467C
:100180003A46334601B0F0BD10B5202A04DB0846DC
:10019000203AD040002110BD0B46D340D04020244F
:1001A000A21A91400843194610BD03460B439B0712
:1001B00003D009E008C9121F08C0042AFAD203E0DC
:1001C0000B780370401C491C521EF9D27047D2B202
:1001D00001E00270401C491EFBD270470022F6E786
:1001E00010B513460A4604461946FFF7F0FF2046AD
:1001F00010BD0321001D401E037812021A43491E40
:10020000F9D510467047F0B51FB40646002082B0FD
:1002100005464024019100901BE0019922460F46BB
:100220003046FFF7B1FF049A059B801A994110D31D
:1002300010461946224600F029F8361A8F410197D8
:10024000224601200021009F00F020F838184D417F
:1002500000902046641E0028DFDC019B00982946A0
:10026000324607B0F0BD0000064C0125064E05E001
:10027000E36807CC2B430C3C98471034B442F7D3C7
:10028000FFF71CFF185700083857000810B5202A40
:1002900004DB0146203A9140002010BD914020230C
:1002A0009C1A0346E3401943904010BDF0B51C4A28
:1002B00090684007C00F31D1106C1B4D81B21948B6
:1002C0001A4B04690120E607002E0AD09982184CC7
:1002D000184B2846A14201D2012100E000211960FB
:1002E00012E0A54306D0144DA54306D0134DA543F7
:1002F00006D009E01983124806E01984114803E08A
:1003000059841149498BD9834103490B9162916802
:100310000E4B1940091D9160024908610020F0BD93
:10032000002401400000002000010020DC12002019
:1003300098080000C00000200000014000000244B6
:10034000000001C0000002C4A0F7FF1FE8FFFF7F0C
:10035000F0B51C4C85B025691B4E6D1C25613768B6
:10036000B668029600976E46758001903181728161
:100370000393206A01011548091800200A5CFF2A2E
:1003800004D01022304600F029F906E0401C102865
:10039000F4D31022304604F07FF9206AE061401C5B
:1003A00020620001012109031030884201D9002098
:1003B0002062E0680649401CE0604867002005B004
:1003C000F0BD00009C000020E456000800D00008AA
:1003D0005C120020002911D08268521882604368A4
:1003E000934200DCD21A00238361C368934201D197
:1003F0000123436182600269521802610846704716
:10040000FCB51D4801901E4D0020E860EA692B698B
:1004100094466A6900922A6AAD69184C0146AE4654
:1004200013E0665B174FBE420ED12E197588401C33
:100430009D4204D9726800922B468C464A1C019E4C
:10044000B54201D28E460195491C01260D013603A5
:10045000B542E6D30A490B616346CB61009B4B6111
:100460000A62C860734612018B61334610329A42A9
:1004700001D900220A62FCBDFFC99A3B00D00008E6
:100480009C000020AA55000010B50421054800F08A
:10049000C6F8054800218161C1610161C160016246
:1004A000084610BD00D000089C00002070B5234C09
:1004B000E06A401CE062224E30688006C00F11D016
:1004C0002068216B40182060216B2046583005467B
:1004D00000F058F820207060A86900280AD0002099
:1004E0002063607230688005C00F02D00120400296
:1004F000706070BD284600F07FF912494A78B35801
:100500005B085B00B350EB682A684D78D2180C4B3F
:100510000C33EA500A4A4B78121D9D582D0C2D04BD
:1005200005439D504978725801231A437250206345
:1005300005488168802211438160D3E7FC010020D7
:1005400000000240F9560008003801400B48C16A1B
:10055000491CC1620A490A689204D20F05D00122DF
:1005600052034A6000220263427208688003C00F8F
:1005700002D0012040044860704700009002002033
:100580000000024010B5002910D0C268436852181C
:10059000934200DCD21A00234361C2608468944213
:1005A00004D1012282618360C360C361084610BD2B
:1005B000FF2109220131D206002801D09162704743
:1005C0009161704701218902034A002801D091629C
:1005D000704791617047000000040048F0B585B095
:1005E00016460D46074600F06DFA012002900020E5
:1005F0000090019503A9684600F0CCF90024760824
:1006000007E060003A5A41190023012000F01CFA6B
:10061000641CA642F5D800F00DFA05B0F0BD7FB518
:100620000D46044600F04EFA00206A4631C203A986
:10063000684600F0AFF900F0FDF904B070BD0000AD
:1006400006490020C861064801690422114301617E
:10065000016940221143016170470000B816002073
:1006600000200240064A0021D16106490A6902239E
:100670001A430A61486108694022104308617047C3
:10068000B81600200020024010B5054B0022DA61A8
:10069000044A1369012423431361018010BD000043
:1006A000B81600200020024010B50B4A0020D16887
:1006B000CB060A4904D5C86902231843C861102033
:1006C000D3685B0705D5CB6901242343CB610421A3
:1006D0000843D06010BD000000200240B816002082
:1006E00070B5054600F000FA0646104C0AE0681C9A
:1006F00008D0002D04D000F0F7F9801BA84201D9E2
:10070000032070BDE068C007F1D1E068800601D524
:100710002020E060E068C00602D4E068400703D50E
:10072000FFF7C2FF012070BD002070BD0020024015
:100730000A07120F01219140014201D001207047A8
:10074000002070470A07120F01219140014201D099
:100750000120704700207047F8B50A05120E254B9E
:100760005200D21809239B01D31800930523DB0103
:10077000D618012305469B020C07D7180020240F2A
:100780002B0003F0C3FF09060A0E12191D21282FA2
:100790002E00FF2928D800981BE0FF2924D80098B4
:1007A00008E0FF2920D8B08A18E080291CD20F2049
:1007B00080011018808E11E0802915D2B88A0DE0D2
:1007C000402911D2B08E09E040290DD20B208001C2
:1007D0000EE0808A02E0802906D2B88E2146FFF71B
:1007E000B1FFF8BD802901D30020F8BD0920C00168
:1007F0001018EEE7DC0C0020C1688268914201DA33
:10080000501A7047914202DC4269002A02D04068C7
:10081000401A704780690028FBD000207047C268EA
:100820008168914201DA501A7047914202DC826974
:10083000002A02D04068401A704740690028FBD067
:100840000020704706490122896912030818010136
:10085000914201D3FF380138024900014018704726
:100860009C00002000D0000800B5082000F08AFDA0
:1008700000BD0000F0B5334B4A00D2180923DB015C
:10088000D4180B230546DB010020D318892D25D071
:100890000EDC2C4F2C4B4E00F619F618803D2B0029
:1008A00003F034FF091F1F152125292E333A1500A7
:1008B0008D2D3FD00CDC8A2D33D08B2D35D08C2D57
:1008C00005D140293ADA0B2080011018808EF0BD46
:1008D000992D03D0A12D01D0FE2DF8D180292DDA3C
:1008E0002EE00846F0BD102928DAB08AF0BD1029A4
:1008F00024DAB08EF0BD102920DA0520C00108E00E
:1009000008291BDA0F208001DFE7082916DA012009
:1009100080021018808AF0BD80290FDA3420205E12
:10092000F0BD80290ADAA08AF0BD402906DA0D2040
:100930008001CAE7402901DAA08EF0BD0020F0BD99
:10094000988EF0BDDC0C00204002000010B5074876
:100950008168074B9A698468A14201D081689A69CD
:10096000044842431014081A10BD0000180000206B
:1009700000E000E05505000031B500F0B5F8009C3E
:100980000546601C00D0641C00F0AEF8401BA0427D
:10099000FAD338BDF8B5054623480F46017E012637
:1009A00001290BD0012101762868204C012807D0AD
:1009B0002046FFF795FE002813D030E00220F8BD56
:1009C0002046FFF78DFE002829D1FFF739FE20468B
:1009D000FFF786FE0646164801690422914301612D
:1009E0001DE00020C04338606C6812E02046FFF72D
:1009F00039FE0E48FFF774FE06460D4802690221D3
:100A00008A430261002E01D03C6008E00120800290
:100A10002418A868810268680818A042E6D802482D
:100A2000002101763046F8BDB816002050C3000002
:100A30000020024003480169802211430161002027
:100A40007047000000200240F0B51FB407461A4866
:100A50000024017E15461E46012907D0012101769A
:100A60001648FFF73DFE002803D020E0022005B025
:100A7000F0BD012F02D0022F00D00427220128460A
:100A80003146FFF781FB81B2019862001018FFF731
:100A9000FBFD0A48FFF724FE09490A695208520083
:100AA0000A61002803D1641CE4B2BC42E6D30249C7
:100AB00000220A76DBE70000B816002050C30000D1
:100AC0000020024005480169090605D50449416036
:100AD0000449416000207047012070470020024017
:100AE00023016745AB89EFCD0148006870470000DE
:100AF000F800002002480168491C016070470000AE
:100B0000F800002010B5064801681022114301606A
:100B1000002000F007F800F017F8002010BD0000DA
:100B20000020024010B5044600F03EF97D21C900C6
:100B3000FFF7DAFA00F06AFB00222146501E00F0AF
:100B400025F8002010BD000008B50F48816901227A
:100B500011438161816911400091C26901040A4316
:100B6000C261C0690022084000901146501F00F089
:100B70000DF800221146901E00F008F800221146E0
:100B8000501E00F003F808BD0010024010B502F03E
:100B900089FB10BDF8B505460068354CC00352D539
:100BA000E0690026C00007D4E16920040143E16147
:100BB000E1690140012600912E480168C90510D461
:100BC0000168821511430160FFF78EFF074604E0BC
:100BD000FFF78AFFC01B642824D826480068C00598
:100BE000F6D5206A03273F02384020D06968394093
:100BF00081421CD0206A226AB843012109040A43B9
:100C00002262226A8A4322622062C0070FD0FFF765
:100C10006BFF009008E0FFF767FF0099411A164844
:100C2000814201D90320F8BD206A8007F3D5206AEC
:100C30006968B84308432062002E04D0E1690120AE
:100C400000078143E1612878C00705D0206BA968BF
:100C500080088000084320632878800605D5206B33
:100C600010218843E968084320630020F8BD000094
:100C7000001002400070004088130000F8B50546DF
:100C800044480E460068C007C00FB0420AD241482F
:100C9000016849084900314301600068C007C00F7E
:100CA000B0425CD128783C4C800705D56068F021C3
:100CB0008843A968084360602878C0073FD0686807
:100CC000012813D02168022813D08907002946DAA9
:100CD00061688908890001436160FFF705FF696861
:100CE000074601290DD0022917D024E02168890385
:100CF000ECE78901EAE7FFF7F7FEC11B27488142CD
:100D000017D860680007800F0128F4D117E0FFF7BB
:100D1000EBFEC11B214881420BD860680007800FA1
:100D20000228F4D10BE0FFF7DFFEC11B1B48814214
:100D300001D90320F8BD60680007800FF3D1154882
:100D40000168C907C90FB1420BD9016849084900B8
:100D5000314301600068C007C00FB04201D00120DC
:100D6000F8BD2878400706D5606807210902884346
:100D7000E9680843606000F01DF86168084A0906E8
:100D8000090F515CC840074908600020FFF7CAFE00
:100D90000020F8BD0020024000100240881300002F
:100DA000FE560008F400002001480068704700006B
:100DB000F400002010B512A30FCB88B06C460FC40E
:100DC00013A30FCB0FC416494A680C2013460340E7
:100DD0001448042B0FD0082B0DD193021B0F6C4627
:100DE000E45CC96A04AB0907090F595CD20304D556
:100DF000FFF77AF9604308B010BD0B486043FAE78B
:100E000002030405060708090A0B0C0D0E0F10104B
:100E10000102030405060708090A0B0C0D0E0F104A
:100E20000010024000127A0000093D00FEB50446A1
:100E30000078D04DC00747D068680007800F0128B0
:100E400007D068680007800F022809D16868C003CE
:100E500006D52868800337D5606800287ED033E047
:100E6000012062680004012A11D08100002A01D00B
:100E7000052A10D02A6882432A602868884328609F
:100E80006068002814D0FFF72FFE06460CE02968A2
:100E900001432960F4E72A680A432A60F7E7FFF76D
:100EA00023FE801B64286FD828688003F7D50BE0E9
:100EB000FFF71AFE064604E0FFF716FE801B6428C3
:100EC000F1D828688003F7D420780126800700280D
:100ED0003BDA68680007800F07D068680007800F5A
:100EE000022809D16868C00306D42868800715D590
:100EF000E068012832D111E0E0680028286815D0A8
:100F000030432860FFF7F0FD074604E0FFF7ECFDF3
:100F1000C01B0228C7D828688007F7D52868F821A1
:100F200088432169C900084328600EE0400840005A
:100F30002860FFF7D9FD074604E0FFF7D5FDC01B89
:100F40000228B0D828688007F7D42078000724D575
:100F5000E0690028686A10D0304300E008E1686268
:100F6000FFF7C2FD074604E0FFF7BEFDC01B0228E5
:100F700099D8686A8007F7D50FE04008400068629A
:100F8000FFF7B2FD074605E09DE0FFF7ADFDC01B92
:100F9000022888D8686A8007F7D420780427400799
:100FA000002860DA00200190E869C00008D4E969EF
:100FB000B8060143E961E96901400120009101900F
:100FC0006D480168C90511D401688215114301609B
:100FD000FFF78AFD009005E0FFF786FD0099401AB3
:100FE000642870D864480068C005F5D5A068012859
:100FF0000AD0002801D0052810D0286A40084000F7
:101000002862286AB84301E0286A30432862A06851
:10101000002812D0FFF768FD00900AE0286A3843E4
:101020002862F1E7FFF760FD0099411A53488142B9
:1010300049D8286A8007F5D50DE0FFF755FD0090E7
:1010400006E0FFF751FD0099411A4C4881423AD819
:10105000286A8007F5D40198002804D0E9690120A6
:1010600000078143E9612078C00635D56069012811
:101070000CD0401D686B23D038436863686B400810
:1010800040006863FFF730FD064622E0686B384396
:101090006863686B30436863FFF726FD064604E02B
:1010A000FFF722FD801B02285BD8686B8007F7D50D
:1010B000686BF8218843A169C900084368630BE0A5
:1010C000B8436863F4E74CE0FFF70EFD801B02288D
:1010D00047D8686B8007F7D4206A002846D0696833
:1010E0000907890F022943D00126360602282868FD
:1010F00005D0B0432860FFF7F7FC044633E0B04367
:101100002860FFF7F1FC074604E0FFF7EDFCC01B89
:10111000022826D828688001F7D4E86AE16A000925
:1011200000010843E862616AA06A084369683D22D9
:101130001204914308436860286830432860FFF731
:10114000D3FC044604E0FFF7CFFC001B022808D8BC
:1011500028688001F7D509E0FFF7C6FC001B0228CC
:1011600001D90320FEBD28688001F5D40020FEBD12
:101170000120FEBD001002400070004088130000F6
:10118000042204490428086902D09043086170478A
:101190001043FBE700E000E015480168643101609E
:1011A00014480168491C016013480168491C01602A
:1011B0001249134AC868401CC860904216DB0020E0
:1011C000C8601048816D491C8165016D491C01652D
:1011D000416D491C41650C48018B002906D0491E10
:1011E00089B20183782901D97821018370470000F1
:1011F000200000201C00002068000020CC000020FF
:10120000102700005C12002090140020094910B53E
:10121000401E884201D9012010BD074C60610321A6
:10122000081F02F03FF80020A06107202061002085
:1012300010BD0000FFFFFF0000E000E010B5FFF769
:10124000ABFF10BDFEE7000010B500200F4A0146BD
:1012500050604B009B18491C1881FF29F9DD0021C3
:1012600005230B4ADB014C00A418E418491CA0829A
:101270001029F8DB00210923DB014C00A418E41835
:10128000491CA086FF29F8DD002010BD540A00206B
:10129000DC0C002010B5402802DB0020C04310BD4C
:1012A00010221143C200094B4000D218C018582424
:1012B0000D23A1529B010021C3189986E300C01899
:1012C0008186034800685065084610BDDC0C00208C
:1012D000F800002070B504461E463830049D03F027
:1012E00001FD20462A463146583003F0FBFC002021
:1012F00070BD000070B5104D064601462846FEF749
:1013000009FF0E4C6061FFF74FFD2946FEF7ECFE2A
:10131000E0600B48314600680546FEF7E5FE2061B7
:101320002A46002307480F21FEF708FF2080606946
:101330006430A060002070BD40420F001800002003
:10134000F40000200000404230B5002372B61022A5
:101350000921C9068A628A61441E0122A240084C02
:10136000002809D025682D0600D4134320258D625E
:1013700052088D61401EF5D162B6184630BD00009E
:1013800010000048F8B572B610220921C9068A6219
:101390008A61C217520F1018C71000200B4E009020
:1013A0000FE000228024082335686D0600D4224314
:1013B00020258D6264088D615B1EF5D16B461A5441
:1013C000401CB842EDDB62B60098F8BD1000004842
:1013D000034610B50020024602E09C5C6040521CAF
:1013E0008A42FADB10BD0000F8B508460D460978C0
:1013F000552901D0252903D0012A01DD451C521EA3
:10140000344C602661792B787143334E8919334E01
:10141000252B30D0B3685B1CB360CB695B1CCB6100
:10142000A17800290FD0E17800290FD001292C499B
:1014300013D007231B02C9180A7501462948FEF775
:10144000B4FE0020E0700020C043F8BD2549264BC3
:1014500055390A750146224807E037235B01C91850
:101460000A750146204B1E482033C018FEF79DFE2A
:10147000E078401CE6E76F79802F06DDF068401CBD
:10148000F060086A401C0862DDE73B4608339A4278
:1014900008D2086A401C0862F068401CF060022014
:1014A000C043F8BDB91DFFF793FFE919897981425F
:1014B0000DD03069401C306161796020414306489D
:1014C0000818416A491C41620320C043F8BD00204E
:1014D000F8BD00004C00002044050020100300204F
:1014E000DC0C0020F1130020D5060000F8B50E46F4
:1014F00005462527079C089906982F706A70AE70DC
:10150000EB7028712746002008372E19372B1AD088
:1015100009DC1A46303A130003F0F8F807261515CF
:10152000262626172600612B0DD006DC382B0AD084
:10153000412B08D0422B17D105E0622B03D0632B3F
:1015400001D0642B10D16C7102E06C71002C03D0BF
:101550002246A81DFEF729FEA11D2846FFF738FFE9
:10156000B0710D20F0713846F8BD0000F1B584B0BF
:10157000FFF7BAFA0546FFF7E9F9604C0646E0794D
:10158000002806D0207A002803D0E068301A3228DC
:1015900005D8E0687D21301AC90088427ED9207ABA
:1015A000574B00281DD0617960225143554A0120D4
:1015B0005050642058646079401CC0B26071E17A78
:1015C000884208D9A06AA662301AE062A079401C5D
:1015D000A071012060714C48008A4C4F002830D027
:1015E00038E0606A401C606249484168491C4160BB
:1015F000617960200A4642434248944610180269C5
:10160000521C02614269521C4261E779002F02D1EB
:10161000876A7F1C87628769BA4200D9826139482C
:10162000032AC8D900226746C251C82098643948A5
:1016300042544800384941180F208001081882861A
:10164000B9E7FFF711F9354980B28882C1B2F98252
:10165000000A38832F49B87D10314870387E887071
:1016600062792F488B5C037089184978417060213A
:1016700013464B4323490027C9588170C770057131
:101680002B0A43712B0C83712B0EC371E6606E46DF
:101690003378A6799B089B00B60700E028E0B60FD8
:1016A00033436E463370002925D0EF210B40337051
:1016B0000290082117480093019141230021203016
:1016C000FFF714FF134902462031049802F04CFB47
:1016D0006179602041430B4808184168491C41600A
:1016E000C268E1688A1A4263C1606563E771277264
:1016F000002005B0F0BD10210B43D8E74C000020BE
:101700005C1200204405002090140020DC10002012
:101710001003002024040020DC0C00201C0F0020FB
:1017200044080020F7B5087886B00C46552801D04B
:10173000252802D0012A00DD4C1C4C4D60796979C6
:101740006022049151434A4A2B4689188A682F46E1
:10175000521C8A60464A803A03921B6BFF68E67807
:10176000DF1B2B46A2789B69303E0093330002F0CA
:10177000CDFF13420B1742424229424242424242AB
:10178000424242422C4542003A49A3798B54227985
:10179000A11D32230092029101900021049A22E0BF
:1017A0006F610098874200DDAF613248A3798354AE
:1017B0000020CF624861086BB84200D20F6301205D
:1017C000287218E00120E87115E02A49A2790A7010
:1017D00010310978A1712279A11D00920291019026
:1017E0004223297900220398FFF780FE02460399DD
:1017F000069802F0B9FA002009B0F0BD6F610098B8
:10180000874200DDAF611B49A079885451001A4A14
:1018100089180F229201891888861848008A0028A2
:1018200009D11748C18E008F00020818154980B2EF
:10183000888602F02BF96A7960214A430C4900201E
:10184000561870616869F062316B814200D2306372
:101850002046677A0A30FEF7CCFC617B0002000A62
:1018600009060843B90071188863A8E74C000020F6
:101870004405002024040020DC0C002090140020EB
:101880009C1000201C0F0020F7B516460D46FFF7F0
:101890005DF81A4C206329780020552903D1012EC8
:1018A00001DD6D1C761E217800290FD00127E7711C
:1018B000324629460098FFF797FD002805D1277288
:1018C000324629460098FFF72DFFFEBD61780029BA
:1018D000FBD00B4C3246A06B2946401CA0630098FD
:1018E00000F012F80028F0D106483246406C20651E
:1018F0002946009800F080F8FEBD00004C00002052
:10190000440500205C120020F0B508460C4609781A
:10191000552901D0252903D0012A01DD441C521E7E
:10192000217800231A4EDB431A4D252906D0A868DA
:10193000401CA860306C401C306409E01449677991
:10194000896C491C802F05DDE868401CE860B164A3
:101950001846F0BD3B4608339A4206D2B164E868A7
:10196000401CE8600220C043F0BDB91DFFF730FD08
:10197000E1198979814208D02869401C2861F06CFE
:10198000401CF0640320C043F0BD0020F0BD000007
:101990004405002010030020F8B5FEF7D7FF1349D7
:1019A0000B690A79002A1FD04C7A114A002C05D005
:1019B0007D20800150640020487215E00C4E0D4CD3
:1019C000C51A8036A54204D97D239B019364012367
:1019D00006E01B19984207D97D239B0193640223DB
:1019E0009367D067086930600020F8BD4C00002084
:1019F0005C120020E02E0000F7B5087884B00C4699
:101A0000552802D1012A00DD4C1C57480168491CA9
:101A1000016066796278554855490390534D0879BD
:101A20008035824208D0FF2A06D0686C401C68646A
:101A30000020C04307B0F0BD824201D0FF2A7DD113
:101A40000A6B00920A6101224A72484AE778A03A7A
:101A5000372F73D007DC303F3B0002F057FE068281
:101A6000138282822482612F7BD004DC382F78D0CD
:101A7000412F76D120E0622F73D0632F71D0642F75
:101A80006FD163E0A3791370384A903A1278A2714B
:101A9000009A0A612279A11D3223009202910196D7
:101AA0000022014644E00020217936230091019074
:101AB0000246029001213BE0A0791070E37AA27AFD
:101AC0001B022B49D218CA6101F0E0FF2848877A2F
:101AD000FEF7CAFE254990390870A071B8006772F8
:101AE0004019018FA172018F090AE172816B090C03
:101AF0002173806B1E49000E60731D48807A401C64
:101B0000C0B288720A2801D3002088722079694601
:101B10000870C00603D57D201649800188642179AC
:101B2000A01D0290124801960091422301790022E3
:101B30000398FFF7DBFCE96B491C00E011E0E96367
:101B400002460399049802F00FF90AE0E279A079BD
:101B500012028018227A637A12041B06D2188018A7
:101B6000C861002066E7000010030020C4040020C4
:101B70004C0000205C120020034610B500200246F5
:101B800002E09C5C6040521C8A42FADB10BD30B51A
:101B90000D46084609781446252901D0012030BD9C
:101BA000062C01D2032030BD611EFFF7E5FF291985
:101BB0002039C97F814201D0042030BD002030BDD2
:101BC00070B51E4605465523049C05982B70697018
:101BD000AA70EE7001462C712246681DFEF7E5FAE8
:101BE000611D2846FFF7C8FF29194871A01D052E61
:101BF00002DA002E00D1002070BD0000FEB51546AF
:101C00000E460746FFF7C3FF040014D0684604726F
:101C10000420009002A90B4801910278401E01782F
:101C2000EE230948FFF7CCFF02460749384602F089
:101C30009BF82046FEBD2A463146384600F006F89D
:101C4000FEBD000089000020D4080020F7B5F94847
:101C500086B04F7842688260421C15780B792E0955
:101C60008D7836012D072D0F2E431670F24A029201
:101C700000780C460490874201D0FF2F75D1214691
:101C8000E5780931ED488C46332D70D028DCEC49DD
:101C9000182D0A686AD012DC072D20D008DC002D30
:101CA00063D0012D3ED0032D41D0052D7ED15EE0C5
:101CB000112D7CD0162D7BD0172DF7D13EE2232D90
:101CC000EED006DC192D74D0212D73D0222DEDD14C
:101CD0008DE1242DE4D0312D49D0322DE6D1BDE067
:101CE000582D68D012DC542D66D008DC342D6FD00E
:101CF0004F2D6ED0502D6DD0532DD7D16DE2552D77
:101D000069D0562D68D0572DD0D163E2294663396A
:101D100004200B0002F0FAFC09F3F2F1151B4A1043
:101D20004A134A00641D00930194012350E2C549FF
:101D30001820B0E23946C6E2C3490C20ABE2C349E1
:101D4000A9E2C24910395020A5E22B4640E2E179D0
:101D50000020B94A03E023185B7A1354401C8842E0
:101D6000F9DBB54802F03EFCA3E076E2EFE1A279B0
:101D7000617912028918E27989B2882B2DD0892BDA
:101D80002FD08A2B31D0832B34D0842B37D0852B86
:101D90003AD0862B3DD0872B40D08B2B43D08C2B39
:101DA00046D0FE2B1DD0A92B47D006E096E29DE140
:101DB000ACE1ECE1C7E065E226E2B32B41D0992B20
:101DC00042D0A12B45D09C48103840180092B0E179
:101DD00044E0F7E1F2E141E24AE2490009189C4897
:101DE0003AE0490009189B4836E04900091898482C
:101DF000203831E049000918952080002CE0490086
:101E000009189D20800027E049000918A5208000BE
:101E100022E049000918FD2080001DE04900091852
:101E20008B48A03818E049000918DD20800013E035
:101E300049000918BD2080000EE0490009188648B5
:101E40000AE04900854807E0854849000818001D58
:101E5000BCE749000120C0060818B7E7A2796179FC
:101E600012028918E27989B2882B25D0892B27D0D4
:101E70008A2B29D0832B2CD0842B2FD0852B32D0AA
:101E8000862B35D0872B3BD08B2B3ED08C2B41D053
:101E9000FE2B45D0A92B47D0B32B49D0992B4AD044
:101EA000A12B4BD064481038401800226146FEF741
:101EB0007CF90020009024E149000918644840E0C2
:101EC0004900091863483CE0490009186048203877
:101ED00037E0490009189520800032E049000918D0
:101EE0009D2080002DE049000918A520800028E0F1
:101EF00049000918FD20800023E0DBE1CEE1C9E1C3
:101F0000490009185248A0381BE049000918DD2093
:101F1000800003E049000918BD2080000818C4E7CC
:101F2000490009184B48F9E7490009184A48F5E7FC
:101F300049004A48F2E74900494802E049000120C7
:101F4000C0060818B2E7A27961791202891809223D
:101F5000920189B2002B0FD0012B13D0022B1CD081
:101F6000032B20D0042B26D0052B2AD0062B28D0DB
:101F7000082B34D000202AE00B095B00181833E04E
:101F8000012024E00B095B00181811E00A07120F6A
:101F9000012191400840F3D119E00A0952001018BC
:101FA0000522D20120E00A09520010180F229201E6
:101FB0008018808EEAE70A09520010180122920266
:101FC00012E0C90008184030007E4006C00F694684
:101FD0000873012003A9212301910090F8E00A0968
:101FE000520010180922D2018018808ACEE7A27907
:101FF00061791202891889B2002B33D0012B3AD0B3
:10200000022B41D0032B48D0042B4FD04022052B6C
:1020100054D0062B52D0072B5BD0002069460873A2
:1020200000200090034803A9401C0191027822235C
:1020300080E6000088000020D4080020DC0C00208E
:10204000540A00204A560008ACF7FF1F107C000815
:10205000B4040000B4050000B406000044050020EC
:102060005C0C00200B070909490009181B0F95207B
:10207000E279800035E00B070909490009181B0FB8
:102080009D20E27980002CE00B070909490009181E
:102090001B0FA520E279800023E00B070909490006
:1020A00009181B0FFD20E27980001AE00B070909CF
:1020B0001B0F49000918E2798E4812E0C900081880
:1020C0004030018B9143E279D207520E11430183D4
:1020D000A6E70B070909490009188648E2791B0F92
:1020E00080300818194601F063FE99E7002B05D0EF
:1020F000012B00D0DDE602F017F8DAE602F04CF82A
:10210000D7E601907C48E378027813E6A1796079FC
:1021100009024018E179794A80B2002B0BD0784C43
:10212000012B03D0774B9B8A002B04D04000001971
:102130000091019009E640008018F9E7002A01D0DB
:1021400000200860002000901723019040E0002A42
:1021500001D000200860A17960790902401885B299
:10216000E2790020684903E02618767A0E54401C74
:102170009042F9DB6449284602F040FA0020093415
:10218000009001905C48039402781823D2E5A1796D
:102190006079090240185B49C882888A00280BD000
:1021A00000208882574801F0A3FD00200090019094
:1021B000514819230278BDE50120F2E75148038315
:1021C000002002E04F490020088300900190E3784E
:1021D0003246AFE54B4920205DE0A17960790902E4
:1021E00040184A4980B20A18E179121D782801D3B3
:1021F000002105E00B18782B02D97821081A81B24A
:10220000C8B201920090A0E5A17960790902401856
:102210003E4980B20B18E2791B1D782801D30022B9
:1022200005E01118782902D97821081A82B261468E
:102230001846FDF7BAFF0020009001902E48E37881
:10224000027839460298FFF7BBFC024602990698CD
:1022500001F08AFD2D4802F0F1F93CE02B4802F034
:10226000EDF900200090019023485523027861E5A4
:10227000244801F03DFD0020009001901E485623A7
:10228000027857E5032109022148FDF7A7FF002046
:1022900000904EE71F490191009056E5A1796079C1
:1022A00009024018E17980B20D01FEF7CBFAE9B2DC
:1022B000009126E7FEF7E8F80020009001900E4814
:1022C0006523027836E50298FFF77AFC0246029908
:1022D000069801F049FD002009B0F0BD02206946D2
:1022E000087303A901200191EE233246009004995E
:1022F000E9E70000140400008900002000800008C5
:1023000000A0000890140020D40800205C0C0020DD
:1023100044050020D012002070B5FEF771F8164871
:1023200000F098FA154C164D6069A865124881684E
:1023300069658188491C81808088E8640E4801F0C5
:10234000D7FC2068286760686867A068A8670122D2
:102350000C4B1146A86DFDF7FBFF28468030E16865
:102360000160A1694160E16981602169C160216A00
:102370000161002070BD0000901400209C0000202E
:102380005C1200203930000030B583680122134010
:1023900002D00022104630BD8C684B68C9682343C8
:1023A000C468034D2C4021430B43C360F2E7000097
:1023B000C73FFFFF30B583680122134002D00022DF
:1023C000104630BD18C94D6823430C6889682C43FA
:1023D00023430B43C168024C21400B43C360EFE72A
:1023E0003CC2FEFF08B504494A6902434A61496993
:1023F0000140009108BD00000010024008B50449EA
:10240000CA690243CA61C9690140009108BD000060
:102410000010024008B504498A6902438A6189694B
:102420000140009108BD00000010024070B5094E47
:10243000044671182039049D0C34CE7F0830102DCD
:1024400003D03250C87F035170BD3251C97F0B5049
:1024500070BD000024520008044A51182039C97F79
:10246000425852085200425070470000245200085F
:10247000044A51182039C97F425801231A43425057
:102480007047000024520008044A51182039C97FBF
:10249000425802231A434250704700002452000859
:1024A000054B10B559182039C97F4358032424031C
:1024B000A3431343435010BDF4560008054B59186D
:1024C0002039C97F001D0B581B0C1B0413430B50F4
:1024D0007047000024520008054B10B559182039E8
:1024E000C97F4358034C23401343435010BD0000A1
:1024F000F4560008EFBFFFFF054B10B559182039FF
:10250000C97F43588024A3431343435010BD0000A8
:10251000F4560008054B10B559182039C97F4358A7
:102520000324A402A3431343435010BDF4560008F0
:10253000054B10B559182039C97F43582024A343AF
:102540001343435010BD0000F4560008054B10B56E
:1025500059182039C97F43584024A343134343509B
:1025600010BD0000F4560008054B10B5591820396D
:10257000C97F435803242402A3431343435010BD8F
:10258000F4560008F0B500243EE001232A46A3409B
:102590001A4038D04F680668134653435D005D19F2
:1025A000AE435F433E4306604E68012E01D0022ECB
:1025B00005D18F6886685F43AE433E4386600F69EE
:1025C000C668AE431D467D432E43C6604D68022D4E
:1025D00019D1FF2A0AD84E69056A534353431A0199
:1025E000D21A954373431D4305620CE0130A1A4641
:1025F0005A435A435A4313019E1A4D69436A6A4328
:10260000B34313434362641C0A681546E240BCD1DD
:102610004A68012A01D0022A06D1CB6841682A46BD
:1026200091435A43114341600120F0BD10B5044667
:1026300001F09CFA206001F07FFA606001F08AFAF4
:10264000A06010BD014610B5002000290FD110492F
:102650000A6B9207920F012A0AD0022A11D0032A8C
:1026600009D001F083FA01F067FA01F073FA10BDA6
:1026700001F07CFA10BD09688907C90FFAD0054836
:1026800010BD096A8907C90FFAD00120C00310BD27
:102690000010024000127A0010B5036800225B06A9
:1026A000DB0F25D10CC98C681A434B6823431A43AE
:1026B000CB681A430B691A434B691A438B691A4357
:1026C00003680C4C23401A43026042680A4B1A40CC
:1026D000CB681B0C1A430B681A43426001238A69BA
:1026E0005B0308399A4202D1898C89B201610122C7
:1026F000104610BD4000FFFFFBF0FFFFF0B5026881
:10270000194B1A4C984201D0A04203D17025AA431C
:102710004D682A43164D174E174F98420AD0A042D3
:1027200008D0164CA04205D0A84203D0B04201D038
:10273000B84204D103242402A243CC68224302609D
:102740008A68C2620A888262984205D0A84203D091
:10275000B04201D0B84201D1097C01634169012234
:10276000114341611046F0BD002C014000040040BF
:10277000004001400044014000480140002000406A
:1027800041680122D202914341608168082291434D
:1027900081607047FEB5044600680D460026C007FC
:1027A000C00F43D1E9686868AA69084329691143E1
:1027B000084321681E4A114008432060A9686068E8
:1027C000032212039043084360606969A0681211F4
:1027D00090430843A0601748844203D10020FFF7CC
:1027E00031FF06E01448844220D16846FFF71EFFFF
:1027F000029800281AD02968002917D00126AA6952
:10280000F3039A420CD140004A088018FDF76CFC93
:1028100081B20A4808400907490F0143E16005E019
:102820004A081018FDF760FC80B2E0603046FEBD3B
:10283000F369FFFF0038014000440040F0FF000052
:1028400010B580220249FDF7B0FC002010BD000049
:1028500064560008F0B584461948184D836812C8BC
:102860000022184F0AE0A85BB84206D170194088D0
:10287000A04202D904461146531C521C01205601A5
:1028800080028642EFD30E4E01207460B360316047
:10289000002906DB480141192022604601F09CF91D
:1028A00001E061468880B068012140018902203042
:1028B000884201D90020B0600020F0BD00C80008A7
:1028C0009C000020AA5500001FB50B46024604A13B
:1028D000684601F007FF0146684601F00BF91FBD8D
:1028E000201B5B25643B25644800000070B5012077
:1028F0008AB04002FFF78EFD224CA06A03263043C7
:10290000A0622149B0050A68824302430A60A26AB4
:1029100083111A43A2620A68824302430A600025B7
:1029200005950695079505A920460895FFF72CFD06
:102930000120039000950195029569460495204673
:10294000FFF738FDE06804218843E0606069C00853
:10295000C0003043606160680843606060680821BF
:1029600088436060A06817218843C9070843A060B6
:10297000A068C00FFCD1A06804490840401CA060BA
:102980000AB070BD0024014008270140E8FFFF7F26
:1029900010B50120FFF726FD00210A2000F060FCA1
:1029A0000A2000F053FC00210B2000F059FC0B2002
:1029B00000F04CFC10BD0000F0B5012087B04004D1
:1029C000FFF710FD01208004FFF70CFD0120C0047B
:1029D000FFF708FD01208005FFF704FD0126C02058
:1029E000002403256A46049631C20927FF0669467A
:1029F0003846FFF7C7FD8020694631C16946384631
:102A00000494FFF7BFFD93200001009003946946F2
:102A10000196029504943846FFF7B4FD3002B86180
:102A200068026A46049631C269463846FFF7AAFD35
:102A30000F486A46049631C20E4F69463846FFF782
:102A4000A1FD0D48009003946946019602950494F7
:102A50003846FFF797FD0720400300900294039447
:102A60006946019604940548FFF78CFD07B0F0BD58
:102A70000704000000040048EEBC00000008004805
:102A8000084907480860084808600420486007486B
:102A90008860CA685207FCD1086105480860704721
:102AA000CCCC00000030004055550000FF0F000066
:102AB000AAAA0000F0B591B0282106A8FDF78EFB68
:102AC00018216846FDF78AFB01252D032846FFF7EC
:102AD000A1FCA801FFF786FC00240820022603279A
:102AE000039404946A460594C1C269461F48FFF7DF
:102AF00049FD102069460394C1C101200490694634
:102B000005941A48FFF73EFD2020039404946A467A
:102B10000594C1C269461548FFF734FD002119200C
:102B200000F09EFBFF200530079007200002089070
:102B30000694E8100B90099408200A940D940E94C2
:102B40000C9007200A4C0F9006A92046FFF7A4FD21
:102B500060681021884360606068A8432843606013
:102B6000206840210843206011B0F0BD00040048F7
:102B700000300140F0B591B0282106A8FDF72EFBEA
:102B800018216846FDF72AFB0127BF033846FFF7E7
:102B900035FC3801FFF726FC0024781002250326B7
:102BA000039404946A46059461C269461C48FFF781
:102BB000E9FC00970394049469461948029601952C
:102BC0000594FFF7DFFCA803039404946A46059478
:102BD00061C269461248FFF7D5FCFF200530079017
:102BE0000720000208900694099428020A940C9485
:102BF0000D940E940B9007200A4C0F9006A92046C6
:102C0000FFF74AFD60681021884360606068082112
:102C100008436060206840210843206011B0F0BD87
:102C2000000400480038004010B586B01421684602
:102C3000FDF7D4FA1020FFF7E1FB0021112000F08E
:102C40000FFB112000F002FB2F20694608800020B6
:102C500001900848084C02902046FFF74FFD20687D
:102C6000802188432060E06801210843E06006B0CD
:102C700010BD0000E70300000010004070B5012007
:102C80008EB08003FFF7C6FB0320400207900220AE
:102C90000890032000240990012509200A9407A91F
:102CA0000C950B94C006FFF76DFC3A4E10220221E2
:102CB0003046FFF711FC002202213046FFF7F0FBFF
:102CC000002202213046FFF733FC00220221304669
:102CD000FFF73CFC802202213046FFF70DFC00226A
:102CE00002213046FFF740FC002202213046FFF768
:102CF00011FC002203213046FFF7EEFB00220321E6
:102D00003046FFF7CDFB002203213046FFF710FCD1
:102D1000002203213046FFF719FC802203213046B0
:102D2000FFF7EAFB002203213046FFF71DFC0022DB
:102D300003213046FFF7EEFB00211B2000F090FA44
:102D40001B2000F083FA1448694600680090019443
:102D500002940394059406940C20104C0490204691
:102D6000FFF718FD60682905084360606068490046
:102D700003225205904308436060A068491208434B
:102D8000A0602046FFF7FCFC2068284320600EB0BE
:102D900070BD0000000002403400002000380140F7
:102DA00070B58EB01C216846FDF718FA182107A8E7
:102DB000FDF714FA012464042046FFF71FFB2046A8
:102DC000FFF710FB0E20079002200890032001253A
:102DD0000990002409200A9507A90C950B94C006B8
:102DE000FFF7D0FB414E102204213046FFF774FB61
:102DF000002204213046FFF753FB00220421304615
:102E0000FFF796FB002204213046FFF79FFB80224C
:102E100004213046FFF770FB002204213046FFF703
:102E2000A3FB002204213046FFF774FB002205219A
:102E30003046FFF751FB002205213046FFF730FBFB
:102E4000002205213046FFF773FB002205213046A2
:102E5000FFF77CFB802205213046FFF74DFB002267
:102E600005213046FFF780FB002205213046FFF7A1
:102E700051FB00211C2000F0F3F91C2000F0E6F9C2
:102E8000A61EFF21304600F0EBF9304600F0DEF9D7
:102E90001748EE03006800900194029403940C20FC
:102EA00004AA51C2134C69462046FFF773FCA06880
:102EB00021140843A060A068B0433043A06020689C
:102EC0001F21490588430843206020684911884331
:102ED00008432060A068A1140843A0602046FFF7C3
:102EE0004FFC2068284320600EB070BD00000240F7
:102EF000380000200044004000B50846042A02D8EB
:102F00000020C04300BD01787F2902D90120C043C1
:102F100000BD41784906490E1F2902D90220C0434D
:102F200000BD114601F08EFE0028F9D0042000BD3E
:102F3000F7B58EB00F46109A0E98FFF7DDFF002808
:102F400003D00020C04311B0F0BDBC4938780978E7
:102F50003A46884201D00020F5E750785388BA8875
:102F60005DBA56BAB64A02241170507029050A0E8D
:102F70002907090F030001F0C9FB11C60A5995ADD5
:102F8000C7E5C6C6C6C6C6C6C6C6F3F1C600F01DAE
:102F9000C008AB4901908870002041E000200590F6
:102FA0000120049007980027C0000A902EE029070E
:102FB00001222809090FD20295420FD24200A148EE
:102FC0001218092080011018808EFDF7B1FB00282F
:102FD00012D005990498014305910DE042009948EB
:102FE0001018FF308130808AFDF7A2FB002803D043
:102FF000049905980843059004986D1C4006000E3E
:103000007F1CADB20490082F03DA0A98C019B042B1
:10301000CDDB8B4A079905985118C8700798401C5A
:10302000019907908842B9DB64186BE0F01DC00875
:1030300083490190887000202FE000200590012036
:10304000049008980027C0000A901CE02805000E94
:1030500042007C4829071218092080011018090F26
:10306000808AFDF765FB002803D004990598084382
:10307000059004986D1C4006000E7F1CADB20490B4
:10308000082F03DA0A98C019B042DFDB6C48089AAF
:1030900005998018C1700898401C019908908842D1
:1030A000CBDBC1E77200664900208A700FE02B1865
:1030B0005F00644BFF180923DB01FB189B8E470060
:1030C0009C461B0A7F18FB7063463B71401CB04254
:1030D000EDDB16E072005A4900208A700FE02B18D1
:1030E0005F00584BFF1809239B01FB189B8A470080
:1030F0009C461B0A7F18FB7063463B71401CB04224
:10310000EDDBA418641C8AE0002E12D0FF20000220
:10311000864207D14B48520012189D20800010189B
:1031200000F03EFE39464648109AFDF73EF8109AE8
:103130007FE04448520012189D208000101800F0D3
:1031400099FDEFE739797879090201433D486A0032
:1031500012180920C00110188186E3E742E0FFE75A
:10316000F01DC008364901908870002035E03818FD
:10317000C07905900120049000200A900B98C000AF
:103180000D9024E0290701222809090FD202954257
:10319000059B049A07D21A4043002A481B189D2019
:1031A0008000181805E01A40430026481818FF3020
:1031B000953000F009FE04986D1C4006000E049046
:1031C0000A98ADB2401C0A90082804DA0D980A99B2
:1031D0004018B042D6DB0B98401C0B9001998842F6
:1031E000C5DB12E000200EE04100CA19D179127A45
:1031F000090211432A185300124A9B180922D201CE
:103200009A189186401CB042EEDB0D48B978817067
:10321000F978C1703979017179794171241DA1B2B0
:10322000074801F00FFD06490855000A09194870C2
:10323000A21C03490E9800F097FD8CE69400002034
:10324000D4090020DC0C002070470000C106C90E24
:1032500001208840014908607047000000E100E05B
:103260008307FF22DB0E9A408907090E9940002848
:103270000BDA0007000F0838830808489B0018186D
:10328000C36993430B43C3617047830804489B00A1
:103290001B181868904308431860704700ED00E061
:1032A00000E400E08307FF22DB0E9A408907090E45
:1032B000994000280BDA0007000F083883080848F7
:1032C0009B001818C36993430B43C361704783087D
:1032D00004489B001B181868904308431860704707
:1032E00000ED00E000E400E010B501200449C00654
:1032F000486004480168491C016000F005F810BDF1
:1033000000ED00E03000002070B5094CE06F0028AF
:103310000CD0084D084902202A68FEF7B5FA0020B3
:103320002860E0678021044801F0D4F870BD0000F7
:103330009002002040000020A403002010B50648A1
:10334000054B00780021403B5A1840325478491C04
:1033500014700F29F8DB10BD1C0D002010B5084CAF
:10336000084B01220221A06DFCF7F2FF064800F095
:10337000BFFCE06D401CE065A06D2066002010BD24
:103380005C12002039300000901400200248C16D0A
:10339000491CC165002070475C120020F3B5FE4E49
:1033A00089B03068002870D0706800281CD00022D6
:1033B0000D21082000F01EFD00221146082000F01B
:1033C00019FD01221146082000F014FD0020F34FE2
:1033D00001463A184032401C11701028F9DBEF4DBD
:1033E0000024012140358AE20122E1E7A200099888
:1033F000099B805CD31805935A78009201265B885C
:1034000001931B2873D012DC0246030001F07EF901
:103410001B5C7272727272723E3E3E3E3E3E5C5C5D
:103420005CA7A7A73E3EBEBEBEBEBEBE5C003428A3
:1034300070D011DC01461C390B0001F067F918A7A8
:10344000A7A7A7A7A7A7A7A7A7A745454545454558
:10345000454545454545FC453A2873D008DC0146BD
:1034600035390B0001F052F905E76E56E76E300072
:10347000DC2804D004DC3B28EFD0C82824D128E184
:10348000DD28FCD0FA28F9D123E141E2D01F030066
:1034900001F03CF90E080A10181B1D1A1A1A1A1A04
:1034A0001A20261A287C4AE0FFF748FF00281FD080
:1034B000287C3AE0FFF742FF002816D1287C00283C
:1034C00013D125E000F0D0FA02E22878F7E7FFF701
:1034D00035FF1DE0287C00280AD0002905D007E030
:1034E000287C002804D1002902D0012010E04DE002
:1034F00000200DE0130001F009F9070C050E111B67
:10350000262E0C0000F0B0FA01990098FDF724F97E
:103510002874DDE120E100F0A7FA0CE0287C002807
:10352000E6D001990098FDF717F90028E0D0DCE714
:10353000287C0028DCD001990098FDF70DF90028BF
:10354000D6D1D2E761E1287C0028CED1019900983C
:10355000FDF702F9B3E7287C0028ECD0C5E7102876
:1035600004D0112804D0122AAED10AE02A7C03E04C
:10357000287C0028A8D001220199009800F03AFC8C
:10358000A6E1287C00289FD00022F5E7059902914A
:1035900015380E79030001F0B9F8120A1215181B3C
:1035A0000F1E3E4F5F6F2E7F878B8F93839A00F0A5
:1035B0005BFA13E028748AE000F056FA1EE000F08F
:1035C00053FA2BE000F050FA39E000F04DFA46E0F3
:1035D00000F04AFA53E0287C002876D03046019962
:1035E000FDF748F906460298C1884079FDF742F98F
:1035F000864268D069E0287C002866D03046019970
:10360000FDF738F906460298C1884079FDF732F98E
:10361000864258D159E0287C002856D0304601997E
:10362000FDF728F906460298C1884079FDF722F98E
:10363000864248DB49E0B3E0287C002845D030468C
:103640000199FDF717F906460298C1884079FDF700
:1036500011F9864237DC38E0287C002835D0304626
:103660000199FDF707F906460298C1884079FDF7F0
:1036700001F9864227DD28E0287C002825D0304645
:103680000199FDF7F7F806460298C1884079FDF7E1
:10369000F1F8864217DA18E0287C002813D19DE75C
:1036A000287C00280FD1A9E7287C00280BD1B5E79A
:1036B000287C002807D1C2E7287C002803D1CEE768
:1036C000287C0028DBD0012074E7002072E7022666
:1036D000FEE00599164609790091C8280CD0DC282F
:1036E00021D0DD2827D0FA28F1D1F000C0194030D0
:1036F000007EC00627D507E0F000C0194030007EEC
:10370000C00601D400211FE0287C002820D00199A8
:103710000098FDF7AFF80146304600F0B3FA3046A6
:1037200000F0FAF846E7F000C0194030007EC0060D
:10373000EAD4012108E0F000C0194030007EC00644
:10374000E2D4022100E003213046FDF7A3FDDBE7D0
:10375000304600F041FDE2E7059902260979009123
:10376000342802D0372816D108E0287C002812D04F
:1037700001990098FDF77EF8401C07E0287C00289E
:1037800009D001990098FDF775F8401E024601998D
:10379000009800F0A5FB9BE0540A0020DC0C002000
:1037A000059933280A7900924A790392C9880291CF
:1037B00014D035281BD0382889D1287C002886D001
:1037C0001046FDF757F8064601990098FDF752F8A4
:1037D000321A0299039800F083FB78E7287C0028CE
:1037E000FBD001990098FDF745F80246F1E7287CE7
:1037F0000028F2D001990098FDF73CF8064602999E
:103800000398FDF737F83218E3E7059936280A7967
:103810004B790593CB8807934B7A0393498902919F
:1038200006D0392812D03A2820D03B284FD132E098
:10383000287C00284BD010460199FDF71BF806465E
:1038400007990598FDF716F832180CE0287C002837
:103850003DD010460199FDF70DF8064607990598E9
:10386000FDF708F8321A029903982EE0287C002808
:103870002DD010460199FCF7FDFF06B20799059877
:10388000FCF7F8FF00B2464332460299039800F075
:1038900027FB321416E0287C002818D01046019926
:1038A000FCF7E8FF06B207990598FCF7E3FF01B2C1
:1038B0003046FCF72FFC02B20E460299039800F046
:1038C0000FFB324602990398491C00F009FB0326BE
:1038D000201141000F48230708181B0F01210289FE
:1038E00099408C46114000D001212B7C0830002BE0
:1038F000634601D01A4300E09A430280A4190A9853
:10390000844200DA72E503484168491C41600020A6
:103910000BB0F0BD540A0020FEB50746402802DB7C
:103920000020C043FEBD2C48F9000E18009640361A
:10393000348BE10601D40020FEBDA1063CD5610612
:103940003FD42649096800980A25406D0190081A5D
:10395000A1070FD0A107890F012905D0022905D0A1
:10396000E143890705D005E0642503E07D25ED00EE
:1039700000E01B4DA84224DB2946FCF7CBFB0146A7
:1039800015487A0012180B20800110188446808E8A
:10399000019B401869435B18009980B24B650D216B
:1039A00089015118898E814203D8084640210C4371
:1039B00034836146888604E0600602D54020844353
:1039C0003483307EB9B24006C20F052000F012FAEF
:1039D000307E4006C00FFEBDDC0C0020F800002049
:1039E00010270000F7B50546FCF719FF04460299B9
:1039F0002868A142A96806DC4018029A0199FCF7E0
:103A0000D4FB029919E0401822460199FCF7CDFB3E
:103A100021462846FCF7DEFC2846FCF700FF064658
:103A20000298071BB7420DDCA96828683A4640187F
:103A300001990919FCF7B9FB39462846FCF7CAFC7D
:103A40000298FEBD002E0CDDA96828683246401899
:103A500001990919FCF7A9FB31462846FCF7BAFC85
:103A6000A4192046FEBD0000074A0F2011183F236D
:103A70005B5C4031401E0B700028F7DC024940318E
:103A8000087C087070470000DC0C002000B500F0D6
:103A900001F800BD70B572B60122134B12039A6192
:103AA0001249040A0C7300248D68AD07ED0FFBD09A
:103AB0000F4D6C62002400E0641C8E683606F60F21
:103AC000FAD1087388688007C00FFBD000206C62B1
:103AD00000E0401C8C682406E40FFAD1E8629A6288
:103AE0009A6162B670BD00000004004800380040D2
:103AF000DC12002010B50C460A4601460348FFF7C9
:103B000071FF00F0CFFC204610BD000054020020E1
:103B100010B50C460A4601460348FFF763FF00F064
:103B2000C1FC204610BD00005402002010B50C4618
:103B300000F020FD204610BD04494968F0221140E4
:103B4000034A0909515CC840704700000010024058
:103B5000FE56000803494968034A4905490F515C6C
:103B6000C8407047001002400E57000810B50648C4
:103B700041680C200140054805D0042903D00829DC
:103B800001D100F005F810BD0010024000127A00CB
:103B900010B50C4C6168012212040B48114002D090
:103BA000914200D14000E16A0907090F491CFCF766
:103BB0009BFA61680F2292041140890C891C4843CA
:103BC00010BD00000010024000093D0000B50820B3
:103BD000FDF7BAFBC0B200BD70B5D4170346A40F01
:103BE0000020A418A41003E085004E595E51401C2B
:103BF0008442F9DC6000D40FA418641003E045008F
:103C00004E5B5E53401C8442F9DC104670BD00B52B
:103C1000FFF7DCFF00BD0000F8B500228024D2438E
:103C2000114D00218C4623464B435B191F880F4ED4
:103C3000B74209D17E26F75A0D4EB74204D15B88B0
:103C4000634501DD0A469C46491C0829EBDB082A2E
:103C500005D2624351198022FFF7BEFF01E0FEF753
:103C6000EFFD0020F8BD000000C00008AA550000CC
:103C7000A55A00000B0702881B0F012199408A43B7
:103C80000280704730B5402802DB0020C04330BDC1
:103C90000D4BC200D21814464034257EAD0611D417
:103CA0004000C0180D239B01C31899860B230021E7
:103CB0009B01C0188186054800685065208B202133
:103CC00008432083002030BDDC0C0020F8000020D9
:103CD00010B500F001F810BD03488168C907C90F8D
:103CE00000D0C068704700000030014070470000FD
:103CF00010B5184C6168491C616017490180A188A2
:103D000041801649CA6C8280496D8160112181838E
:103D10001349C183A1684A011249511800228B5CE2
:103D2000FF2B03D02022FCF759FC05E0521C202A6F
:103D3000F5D3202200F0B0FCA0682060401CA060F9
:103D40004001012189022030884201D90020A06071
:103D5000002010BD9C000020AA5500005C1200202D
:103D6000A55A000000C8000810B514460A460128EC
:103D700002D0022806D00DE021461046FFF7C8FE0B
:103D8000054804E021461046FFF7D0FE0348816F46
:103D9000491C8167204610BDFC01002090020020D4
:103DA0000B0702881B0F012199400A4302807047CC
:103DB0000907090F01238B400188002A01D019430C
:103DC00000E099430180704710B5002A02D0FFF748
:103DD000E7FF10BDFFF74EFF10BD0907090F0123D4
:103DE0008B400188002A01D0194300E099430180EB
:103DF0007047000070B50B051B0E204C5B000D07D3
:103E00001C192D0F030000F081FC09060B14191E6C
:103E100022272C313600FF292DD89520800003E081
:103E2000FF2928D89D20800020182946FFF7D5FFBC
:103E300021E0FF291FD8A5208000F5E780291AD2AC
:103E4000FD208000F0E7802915D20D48ECE74029DD
:103E500011D2AD208000E7E740290CD2B5208000C8
:103E6000E2E7802907D206482030DDE7802902D228
:103E700003488030D8E7002070BD0000DC0C002033
:103E8000140400000121C903034A002801D09162F3
:103E900070479161704700000008004801218903C4
:103EA000034A002801D09162704791617047000079
:103EB0000008004801210922C902D206002801D0C9
:103EC000916170479162704701214903034A0028BC
:103ED00001D091627047916170470000000800486E
:103EE000F0B5304C4B001C190923DB01E6180B23FD
:103EF000DB01E51892B28A283DD00EDC294F4B0039
:103F0000DF1909239B01FF188338030000F0FEFB33
:103F10000714181C21262D46480099283ED006DC9F
:103F20008B282CD08C2831D08D2839D133E0A12892
:103F300034D0FE2834D131E0102931DABA822FE0B2
:103F400010292DDABA862BE0102929DA0520C001C4
:103F500008E0082924DA0F20800114E008291FDA7C
:103F600001208002201882821AE0802918DAB286A5
:103F700016E0AA8614E0802912DAB28210E0402905
:103F80000EDA0D2080012018828609E0402907DA28
:103F90000B208001F7E7402902DAE8E78029E8DB17
:103FA0000020F0BDDC0C0020F0B591B0002600F040
:103FB00009FEFCF7CBFC07901021394800F062FEA7
:103FC0000A90FCF7C3FC04901021354800F006FE6F
:103FD0000990FCF7BBFC03901021314800F01AFE59
:103FE0000290FCF7B3FC054610212D4800F02AFE94
:103FF0000190FCF7ABFC2B49044688680122104372
:104000008860901E086128480861254B00201A5CD2
:104010000A70401C1028FADB0F68FCF797FC029925
:1040200002970091214F0890B81921A1099B0A9A83
:1040300000F058FB86190898039A011B601B029137
:10404000019004990398AA1A431A08460799009206
:10405000421AB81920A100F045FB84190BA8FEF7FD
:10406000E5FA264842680120000402403819134648
:1040700023A100F037FB0419381926A10B9A00F090
:1040800031FB01193846FFF735FD01210D20FEF700
:104090001BFC244903208860002011B0F0BD000003
:1040A000145200080030024001A00000FC00002073
:1040B0000D0A435243202025303458202025303427
:1040C00058202025303458202025303458202025F1
:1040D0003034580D0A00000074696D6520253034B5
:1040E00064202025303464202025303464202025AD
:1040F0003034642020253034640D0A000010024062
:104100004D61696E536F7572636520257820256453
:10411000200D0A00737973636C6B202564200D0AEF
:10412000000000000000002030B5002317491846A9
:104130004B6042005218401C1381FF28F9DD002219
:1041400005241348E40155002D182D19521CAB828B
:10415000102AF8DB00220924E40155002D182D193E
:10416000521CAB86FF2AF8DD00221024D3001B1856
:1041700040331D8B521CA5431D83402AF6DB0120D2
:10418000086004494882002030BD0000540A002025
:10419000DC0C00209014002010B500220C480923EC
:1041A00002600C4910469B0144006418E418401C4E
:1041B000A2861028F8DB002001239B02440064182B
:1041C000E418401CA2820828F8DB002010BD000083
:1041D000540A0020DC0C002010B5402802DB00202F
:1041E000C04310BD0B4AC10089180B4640331C7EEA
:1041F000A4060DD5400080180B22002492018018DF
:104200008486054800684865188B202188431883F8
:10421000002010BDDC0C0020F800002010B5FCF7D9
:1042200069FCFDF70BF810BD70B594B030216846FD
:10423000FBF7D4FF002501240E952004099000947B
:1042400005200F95C0040D95022601940A900C9547
:1042500008960B946846FCF7E9FD002803D08621F8
:1042600015A000F03DFA07200C900E9501210D9647
:104270000F950CA8FCF702FD002803D092210EA098
:1042800000F02EFA109410A81294FCF783FC00287A
:1042900003D0A12108A000F023FA4B208001FCF7F5
:1042A000B5FF0420FCF76CFF00221146501EFCF7FE
:1042B0006DFC14B070BD00002E2E5C436F6D4C6918
:1042C000625C5372635C4253502E63001348016872
:1042D0000122114301604168114A114041600168A7
:1042E000104A11400160016801229204914301606B
:1042F00041683F22120491434160C16A09090901E2
:10430000C162016BFF22143291430163416B490882
:1043100049004163002181607047000000100240A5
:104320000CB8FF08FFFFF6FE04480169C907C90F72
:1043300002D00121C9430161704700000010004014
:1043400070B51B4CE0698006C10F1A4811D01A4A9B
:1043500001211160194A11600169491C0161A18C98
:104360004268521C4260174B154D1A68A954521CE2
:104370001A60E1690907C90F04D008212162C169E7
:10438000491CC1612068C006C00F07D0E069C006A3
:10439000C00F03D01020206200F03CF8E069400616
:1043A000C00F03D04020206200F074F870BD000000
:1043B00000380140FC01002044000020480000209B
:1043C000240300203C00002010B5104CE069E06997
:1043D0000007C00F05D0082020620D48C169491CA4
:1043E000C1612068C006C00F07D0E069C006C00FD9
:1043F00003D01020206200F09DF8E0694006C00F55
:1044000003D04020206200F0E5F810BD00440040D9
:10441000900200200548416A491C4162044909682C
:10442000002901DD0121C16770470000FC01002067
:104430003C000020F8B5144E0C46054602213046DB
:10444000FEF70AF810200090104B2A460221304651
:10445000FDF7ECFF224602213046FEF72FF802213D
:104460003046FEF705F80A48046301214172022133
:104470003046FEF709F80548283881688022114344
:1044800081602046F8BD000000000240283801404D
:10449000FC0100200248016A491C016270470000CB
:1044A000FC01002010B50A48407A00280DD1084CC4
:1044B000206F5834002808D12046FCF79DF90146AA
:1044C000E26820688018FFF7B5FF002010BD0000EB
:1044D000FC010020F8B5144E0C4605460521304677
:1044E000FDF7BAFF002000902B46104A0521304608
:1044F000FDF79CFF224605213046FDF7DFFF052131
:104500003046FDF7B5FF0A48446301218172052159
:104510003046FDF7B9FF0548243881684022114331
:1045200081600020F8BD00000000024024440040EB
:10453000900200200A480B4900794058802180B23F
:10454000091A0948012201600848C267426A521CE0
:104550004262002903DD01200549000748607047D9
:104560002452000804000240400000209002002075
:1045700000ED00E0F8B5144E0C4605460421304627
:10458000FDF76AFF10200090104B2A4604213046A8
:10459000FDF74CFF224604213046FDF78FFF042132
:1045A0003046FDF765FF0A4804630121417204218A
:1045B0003046FDF769FF054828388168802211439D
:1045C00081602046F8BD0000000002402844004001
:1045D000900200200248016A491C016270470000F5
:1045E000900200200A4610B503494B885B1C4380AB
:1045F000FBF7F4FF002010BD007C000870B50C46EE
:104600000B494118002B08D00A4D4519012B03D046
:10461000094B9B8A002B00D129468005204603D0F8
:1046200000F03AF8002070BDFBF7D8FFFAE7000071
:104630000080000800A000089014002070B5418898
:10464000134A491C4180114901807E210A5280246D
:1046500010490022134663435D180023EE5CFF2ED1
:1046600003D0521C082AF5DB0AE05B1CA342F5DBF1
:10467000082A05D262435118802200F00DF802E0AA
:104680008022FBF7ABFF002070BD0000AA550000A0
:10469000A55A000000C00008F7B515460E46FCF705
:1046A00011FA0024AF0808E00099A0000A58811907
:1046B00000230220FCF7C8F9641CA742F4D87C0050
:1046C0006D0808E0009960000A5A81190023012052
:1046D000FCF7BAF9641CA542F4D8FCF7ABF9FEBDAF
:1046E000FEE700000FB410B504A9074B02AA039817
:1046F00000F028F8044602A9002000F05DFA2046E8
:1047000010BC08BC04B01847B94B000830B474465C
:10471000641E2578641CAB4200D21D46635D5B00BD
:10472000E31830BC184702E008C8121F08C1002A6D
:10473000FAD170477047002001E001C1121F002A22
:10474000FBD17047FFB591B00F460546002606E045
:1047500025280AD0149A139990476D1C761C287846
:104760000028F5D1304615B0F0BD00240094012199
:10477000F34A029400E004436D1C2B780846203B6A
:1047800098401042F7D128782A280ED002212878A4
:104790000246303A092A15D8009A0A235A43303A79
:1047A00080180C436D1C0090F1E701CF00900028A9
:1047B00005DA0120400304430098404200900220A3
:1047C00004436D1C28782E2815D1042004436878F2
:1047D0006D1C2A280AD101CF6D1C02900BE00299B2
:1047E0000A225143303940186D1C02902878014646
:1047F00030390929F3D928786C2810D006DC4C28E8
:104800001AD068280ED06A2817D104E0742813D073
:104810007A2812D110E00120400504430CE0012168
:10482000090501E0032109050C436978814203D1A0
:104830000120000524186D1C6D1C287803906E283B
:104840001ED00CDC632831D004DC00288AD0582824
:1048500011D1B2E064287BD069280CD178E07328AC
:104860002DD004DC6F2870D0702804D1A7E0752803
:104870006CD078286BD0149A13999047761C62E01C
:104880006002400F022807D003280AD004283868A5
:104890000AD006603F1D56E03868F1170660416097
:1048A000F8E738680680F5E70670F3E73878694678
:1048B00008740020487404A80390012003E03868BD
:1048C00003900020C0433F1D61070FD5002101E088
:1048D0000199491C029A0191914213DA8142F7DB56
:1048E000019A0399895C0029F2D10BE0002101E0D3
:1048F0000199491C01918142FADB019A0399895C73
:104900000029F5D101990098139A401A0090214688
:10491000149B00F03BF901998019461807E00398B1
:1049200003990078491C0391149A139990470198B0
:10493000401E0190401CF2D12146149B139A00980E
:1049400000F014F986196D1C09E741E033E034E00A
:104950000A200021049005916002410F022905D030
:1049600001CFC2179446032905D007E0FF1DFF08B9
:10497000FF0003CF06E000B2C2179446042902D11B
:1049800040B2C1178C4600226146944506DA0A46B9
:104990000021404291418C462D2102E0210504D5A1
:1049A0002B216A461176012103E0E10701D0202185
:1049B000F7E7019154E00A200BE0102009E01020F5
:1049C000049000210420044308200591029003E094
:1049D00008200021059104906002410F022905D0B2
:1049E00001CF00229446032906D006E0FF1DFF08F0
:1049F000FF0003CF8C4603E080B2042900D1C0B28F
:104A00000021019121072BD50399702906D0049A22
:104A10001021059B4A401A4305D00EE040216A460A
:104A20001176012108E06146014306D030216A4633
:104A300011760399517602210191049A0821059B70
:104A40004A401A430CD16146014301D1610707D5A1
:104A500030216A461176012101910299491E029185
:104A60000399582904D037A103910FA90F910DE0A4
:104A700039A1F9E76146059B049AFBF7C4FB039B48
:104A80008C469B5C0F9A521E0F9213706146014335
:104A9000F0D10F9807A9081A20300390600704D5B9
:104AA000012000048443029801E001200290039950
:104AB000884201DD401A00E0002041180290019870
:104AC00009180098401A0090E00306D42146149B70
:104AD000139A009800F05AF886190020049008E014
:104AE00006A9085C149A139990470498401C761CF8
:104AF000049001998842F3DBE0030CD52146149B16
:104B0000139A009800F042F8861904E0149A3020B5
:104B100013999047761C0299481E02900029F5DCF3
:104B200008E00F980F990078491C0F91149A139977
:104B30009047761C0399481E03900029F1DCFBE6A0
:104B40000928010030313233343536373839616263
:104B50006364656600000000303132333435363727
:104B6000383941424344454600000000F8B5044648
:104B700000251E461746880404D405E03946202047
:104B8000B0476D1C641EF9D52846F8BDFFB5044634
:104B9000002581B01E46C80301D5302700E020273C
:104BA000880404D505E038460399B0476D1C641E9F
:104BB000F9D5284605B0F0BD0A68531C0B6010708B
:104BC0007047000010B50A2101A0FEF793FF10BD49
:104BD0001B5B324A1B5B303B3048000030B503465C
:104BE0000A4800290ED11A78094C50400022C50706
:104BF00002D04008604000E04008521CD2B2082AAF
:104C0000F5D35B1C491EEED230BD0000FFFF000053
:104C100001A0000070B50A4DFF23EE1D1A46F936BB
:104C200005E0047854402A5D5A40335D401C0C4630
:104C3000491E89B2002CF4D11802104370BD000047
:104C40002A54000870B504460C4800220C4E11E0AE
:104C50002578521C2B4643401B07DB0EF35A0009F4
:104C60004340280958400007C00E305A1B095840DD
:104C700092B2641C8A42EBD370BD0000FFFF0000BB
:104C80002A56000810B5084A084B07E0047854403B
:104C90002406E40D1C5B120A6240401C491EF5D23A
:104CA000D04380B210BD0000FFFF00002A52000870
:104CB00010B572B604220A498A614A01131102240E
:104CC0008C62104201D08B6100E08B62520802249A
:104CD0008C61002AF3D104208862886162B610BD1D
:104CE0000004004806C00021016041608160C1608D
:104CF0000122026141610846704700000EB5FE4F77
:104D00000126FF203E830530FC4B80220090991A3B
:104D1000FB48FCF7DFFA4020FA4B0246191A0090D4
:104D2000F948FCF7D7FAFBF7EDFE0021F74A0D46EC
:104D30006020484380184560856005614561856154
:104D4000C561056285624562C562491C0563092922
:104D5000EEDBEF4CEF482567C06A6066EE480068FE
:104D6000A066EE48406AE066FFF75EFAED49EC485F
:104D70000860FCF7BFFAFDF71FFEFDF709FEFDF71F
:104D8000CBFAE948FEF748FFDB480683FEF73FFF12
:104D90000107A063090FE54A6063E54F11701F2802
:104DA00005D0C00606D5E34806703D7005E0E24830
:104DB0000670F8E7DF4805703E70E0480170E04992
:104DC00001200870E120DF4940020860FDF756FF2E
:104DD000FDF7E6FFFDF76EFEDB48416840263143F4
:104DE0004160FDF7C7FEFDF781FDFDF749FEFDF7C8
:104DF0001BFFD6480168012211430160D4480168B5
:104E000020221143016001681022114301600168F2
:104E1000314301608021CF48FFF75CFBCE48016839
:104E20001022114301600168314301600A20FBF741
:104E3000A3FD0120FFF748F80020FFF72FF800201E
:104E4000FEF724FE0120FBF7B3FBC448FFF730FF59
:104E50000120FBF7B7FB0020FFF72CF8FFF7A4F8C1
:104E6000FBF774FD6066A44D002028826882AE487E
:104E7000C0882882288A01280AD1FCF7E5F9208F0A
:104E8000202108406882688A002801D0FFF74CF989
:104E9000B34E5A2070840121B24889024118019111
:104EA0000F218901411802910F21C9014718AE4D08
:104EB0000020287001206870FBF748FD2861FBF78F
:104EC00013FE0090FEF7A3FE05468B48008AC0073C
:104ED0000BD0A806208F04D5800606D4FFF724F94E
:104EE00003E0800601D5FFF757F9A5630098E0635A
:104EF0000920C0060069B8849C480069F8849C4871
:104F0000006938859B4800697885FBF7ADFC80B265
:104F1000B082FFF7CDFEFBF719FD934D686196480F
:104F20000068002801D00020B082206CC006C00EAE
:104F300002281CD1FBF7BAF98F48016800290ED06E
:104F40000021B1828D490A68002A10D100680860EA
:104F50008B4800688B490860FEF700FA07E0874934
:104F60000A68002A03D000680860FEF70FFA62485A
:104F7000008A01280BD16048818A002927D0824904
:104F8000A960C18A81480160A868FEF707FA606ECF
:104F900069696166081AA066E16E884200D2E0661F
:104FA000216F884200D92067FBF7D0FCA8616148D7
:104FB0000078002806D061480078002802D002203E
:104FC000FCF7D4FA0098800403D5012002E0704970
:104FD000D6E7002028700098000501D5012000E0E8
:104FE000002068705248007800281AD00220FCF790
:104FF000D3FC606C002801D16649087065480178CF
:105000000198818264480168890401D5012100E08A
:10501000002129700068000501D5012000E0002072
:105020006870606C002801D0401E6064A06C00288D
:1050300001D0401EA0643048018B002948D0687818
:10504000FEF742FF6878FEF729FF6878FEF71AFF3F
:105050006878002801D1012000E00020FEF72AFF37
:10506000FBF774FCE8610298B18A81860198808A16
:10507000B086FBF76BFC2862B08EFEF707FDFBF7EE
:1050800065FC0A2168620846FBF71EF80220401CF6
:105090004028FCDB206C401C20644048016800294B
:1050A00029DD174AD26F002A25D08AB23C49012057
:1050B000FDF73EFF002805D0384839490268012035
:1050C000FCF79CFD3549002008600D49C86789E060
:1050D000008A012866D0606C002867D06878FEF7E7
:1050E000F3FEA06C002863D06878FEF7D7FE6878DE
:1050F000FEF7C8FEB1E762E09014002030150020F2
:10510000FC010020741600209002002044050020BD
:105110005C12002080F7FF1F3000002000100240CA
:1051200010270000140000205C0C0020500000201C
:105130004D0000204C00002084000020570000207B
:1051400051000020340000200030014000100040D9
:1051500000380140A403002000440040FFFF00008D
:105160001C0F0020DC0C0020CC00002000040048B4
:1051700000080048000C0048C0000020C4000020C7
:105180001C000020C800002000A00008980000209B
:105190000080000824040020680000203C0000205B
:1051A0002403002015480068002898D0287896E746
:1051B0000020FEF773FE0020FEF764FE4BE7104967
:1051C000686888420DD90F484168012212051143D1
:1051D00041604168520003235B05994311434160DC
:1051E00001E0401C686008480078002802D00020D8
:1051F000FBF7C2FB06490548086058E6540A002040
:10520000C0270900003801404D000020AAAA000074
:1052100000300040112233445566778899AABBCCF0
:10522000DDEEFF00081C30445800000089111223F5
:105230009B322446AD573665BF74488CC19D5AAF2A
:10524000D3BE6CCAE5DB7EE9F7F881100801933321
:105250001A22A5562C47B7753E64C99C408DDBBF0A
:1052600052AEEDDA64CBFFF976E802218B30100202
:1052700099132667AF763444BD554AADC3BC588EEA
:10528000D19F6EEBE7FA7CC8F5D983310A209112E1
:105290001803A7772E66B5543C45CBBD42ACD99ECA
:1052A000508FEFFB66EAFDD874C904428D53166136
:1052B0009F702004A9153227BB364CCEC5DF5EEDAA
:1052C000D7FC6888E1997AABF3BA85520C439771A1
:1052D0001E60A1142805B3373A26CDDE44CFDFFD8A
:1052E00056ECE9986089FBBB72AA06638F72144082
:1052F0009D512225AB343006B9174EEFC7FE5CCC6A
:10530000D5DD6AA9E3B8788AF19B87730E62955060
:105310001C41A3352A24B1163807CFFF46EEDDDC49
:1053200054CDEBB962A8F99A708B088481951AA7BD
:1053300093B62CC2A5D33EE1B7F04008C919522B51
:10534000DB3A644EED5F766DFF7C899400859BB7F8
:1053500012A6ADD224C3BFF136E0C1184809D33B31
:105360005A2AE55E6C4FF77D7E6C0AA583B41886D9
:1053700091972EE3A7F23CC0B5D14229CB38500A11
:10538000D91B666FEF7E744CFD5D8BB502A49996B8
:105390001087AFF326E2BDD034C1C3394A28D11AF1
:1053A000580BE77F6E6EF55C7C4D0CC685D71EE50D
:1053B00097F42880A1913AA3B3B2444ACD5B5669D1
:1053C000DF78600CE91D722FFB3E8DD604C79FF578
:1053D00016E4A9902081BBB332A2C55A4C4BD779B1
:1053E0005E68E11C680DF33F7A2E0EE787F61CC459
:1053F00095D52AA1A3B03882B193466BCF7A544891
:10540000DD59622DEB3C700EF91F8FF706E69DD437
:1054100014C5ABB122A0B9923083C77B4E6AD55870
:105420005C49E33D6A2CF11E780F00C1814001C048
:10543000804101C0804100C1814001C0804100C164
:10544000814000C1814001C0804101C0804100C154
:10545000814000C1814001C0804100C1814001C044
:10546000804101C0804100C1814001C0804100C134
:10547000814000C1814001C0804100C1814001C024
:10548000804101C0804100C1814000C1814001C014
:10549000804101C0804100C1814001C0804100C104
:1054A000814000C1814001C0804101C0804100C1F4
:1054B000814000C1814001C0804100C1814001C0E4
:1054C000804101C0804100C1814000C1814001C0D4
:1054D000804101C0804100C1814001C0804100C1C4
:1054E000814000C1814001C0804100C1814001C0B4
:1054F000804101C0804100C1814001C0804100C1A4
:10550000814000C1814001C0804101C0804100C193
:10551000814000C1814001C0804100C1814001C083
:10552000804101C0804100C1814000C0C101C3036E
:1055300002C2C60607C705C5C404CC0C0DCD0FCFEB
:10554000CE0E0ACACB0BC90908C8D81819D91BDB5B
:10555000DA1A1EDEDF1FDD1D1CDC14D4D515D717AB
:1055600016D6D21213D311D1D010F03031F133F35B
:10557000F23236F6F737F53534F43CFCFD3DFF3FAB
:105580003EFEFA3A3BFB39F9F83828E8E929EB2BDB
:105590002AEAEE2E2FEF2DEDEC2CE42425E527E76B
:1055A000E62622E2E323E12120E0A06061A163A3DB
:1055B000A26266A6A767A56564A46CACAD6DAF6F6B
:1055C0006EAEAA6A6BAB69A9A86878B8B979BB7BDB
:1055D0007ABABE7E7FBF7DBDBC7CB47475B577B72B
:1055E000B67672B2B373B17170B05090915193535B
:1055F000529296565797559594549C5C5D9D5F9F2B
:105600009E5E5A9A9B5B99595898884849894B8B5A
:105610008A4A4E8E8F4F8D4D4C8C448485458747EA
:1056200046868242438341818040000001CC01D8FC
:10563000001401F0003C002801E401A0006C007897
:1056400001B40050019C01880044010A07010001D7
:105650000001040108080000000000000000000034
:1056600006000000AA550000000100000000000034
:10567000010001000009000000000000000002001D
:105680000000000900000000000000000000000011
:1056900000000000000000000000000010101010CA
:1056A000101010101010101010101010100020000A
:1056B00030004000500060000300000004000000C3
:1056C00005000000060000000700000008000000C0
:1056D000090000000A0000000B0000000C000000A0
:1056E0001100A55AAA5500000000000000000000AB
:1056F00000000000081C304458081C3044580000CA
:105700000000000000000102030406070809000071
:1057100000000102030400003857000800000020C8
:10572000FC0000002647000834580008FC00002058
:10573000DC190000364700080000000000000000EF
:105740000000000000000000010000001027000021
:105750000000000000000000000000000000000049
:1057600000000000000000000000000000C2010076
:1057700040420F0000000000000000000000000098
:105780000000000000000100000000010101000015
:105790000000000000000000000000000000000009
:1057A00000000000000000000000000000000000F9
:1057B00000000000000000000000000000000000E9
:1057C00001000000000000000000000001000000D7
:1057D00097000000FFFFFFFF000000000000000036
:1057E00000000000000000000000000000000000B9
:1057F00000000000000000000000000000000000A9
:105800000000000000000000000000000080000810
:105810000000000000000000000000000000000088
:10582000000000000000000000000000001BB700A6
:045830000000000074
:04000005080000B53A
:00000001FF
